:0200000480007A
:100000006F00C004732F2034930F8000630AFF0336
:10001000930F90006306FF03930FB0006302FF038A
:10002000170F0080130F0FFE63040F0067000F000F
:10003000732F203463540F006F004000136E9E53E3
:10004000171F00002320CFFD6FF09FFF732540F1A5
:100050006310050073251030635805000F00F00F82
:10006000130E100073000000130E00009702000032
:10007000938282F973905230735020307350303035
:1000800073504030970200809382C2F7638C020065
:10009000739052109302B01A739022307323203061
:1000A000E39E62F873500030970200009382420191
:1000B00073901234732540F17300203097200000B4
:1000C000938040F41301A0FA238020008381000074
:1000D000930EA0FA130E2000639CD13D97200000E0
:1000E000938040F213010000A38020008381100060
:1000F000930E0000130E3000639CD13B972000004C
:10010000938040F037F1FFFF130101FA23812000B3
:1001100083912000B7FEFFFF938E0EFA130E40006E
:100120006398D139972000009380C0ED1301A0009F
:10013000A381200083813000930EA000130E500095
:100140006398D13797200000938030EC1301A0FA18
:10015000A38E20FE8381D0FF930EA0FA130E6000C1
:100160006398D13597200000938030EA1301000096
:10017000238F20FE8381E0FF930E0000130E70009A
:100180006398D13397200000938030E8130100FA80
:10019000A38F20FE8381F0FF930E00FA130E8000E0
:1001A0006398D13197200000938030E61301A000BE
:1001B0002380200083810000930EA000130E900086
:1001C0006398D12F97200000938040E43751341278
:1001D00013018167138200FE230022028381000045
:1001E000930E8007130EA0006394D12D972000007A
:1001F0009380C0E137310000130181099380A0FF93
:10020000A383200017220000130252E083010200A2
:10021000930E80F9130EB000639CD129130EC00019
:10022000130200009300D0FD17210000130181DDAF
:100230002300110083010100930ED0FD639AD127A2
:100240001302120093022000E31E52FC130ED00092
:10025000130200009300D0FC17210000130181DA83
:1002600013000000A300110083011100930ED0FCC5
:100270006390D1251302120093022000E31C52FC6C
:10028000130EE000130200009300C0FC17210000D1
:10029000130141D7130000001300000023011100D7
:1002A00083012100930EC0FC6394D121130212003C
:1002B00093022000E31A52FC130EF0001302000018
:1002C0009300C0FB1300000017210000130181D32D
:1002D000A301110083013100930EC0FB639AD11D6D
:1002E0001302120093022000E31C52FC130E0001C3
:1002F000130200009300B0FB130000001721000060
:10030000130141D0130000002302110083014100BA
:10031000930EB0FB639ED1191302120093022000CA
:10032000E31A52FC130E1001130200009300B0FAFE
:10033000130000001300000017210000130181CCFE
:10034000A302110083015100930EB0FA6392D117FA
:100350001302120093022000E31A52FC130E200134
:1003600013020000172100001301C1C993003003DC
:100370002300110083010100930E3003639AD1130F
:100380001302120093022000E31E52FC130E3001F0
:1003900013020000172100001301C1C693003002B0
:1003A00013000000A300110083011100930E30021E
:1003B0006390D1111302120093022000E31C52FC3F
:1003C000130E40011302000017210000130181C326
:1003D000930020021300000013000000230111000D
:1003E00083012100930E20026394D10D13021200A9
:1003F00093022000E31A52FC130E50011302000076
:1004000017210000130101C0130000009300200118
:10041000A301110083013100930E2001639AD109D9
:100420001302120093022000E31C52FC130E600121
:1004300013020000172100001301C1BC13000000CB
:1004400093001001130000002302110083014100FA
:10045000930E1001639ED105130212009302200037
:10046000E31A52FC130E7001130200001721000062
:10047000130141B9130000001300000093001000A5
:10048000A302110083015100930E10006392D10367
:100490001302120093022000E31A52FC1305F00E1F
:1004A00097250000938505B6A381A500631CC001B4
:1004B0000F00F00F63000E00131E1E00136E1E00CF
:1004C000730000000F00F00F130E10007300000007
:1004D000731000C0000000000000000000000000D9
:1004E000000000000000000000000000000000000C
:1004F00000000000000000000000000000000000FC
:0405000000000000F7
:1010000000000000000000000000000000000000E0
:1010100000000000000000000000000000000000D0
:1010200000000000000000000000000000000000C0
:1010300000000000000000000000000000000000B0
:081040000000000000000000A8
:10200000EFEFEFEFEFEFEFEFEFEF0000000000007A
:040000058000200057
:00000001FF
